:020000003328A3
:10000800F000030E83120313A0000A08A1008A015E
:100018000B1C2A280130C420831203132810851AC8
:100028002814A810051AA81428030319A615831262
:1000380003132808043A03192615831203132811F9
:1000480028182815A811A818A8150B10831203132F
:1000580021088A00200E8300F00E700E090083121A
:1000680003179E019F013030831603138500860114
:1000780087018113151695161616961635308312B4
:100088009000A8012610A614A7012611A611860122
:1000980087118B158F018E018B1783120313261D71
:1000A80063288717BB20831203132611A61C261466
:1000B80083120313A61010108F018E0110148312DF
:1000C8000313A61DAE28261CA0282610A611A618C4
:1000D8009928A70A2708053A0319A70183120313C9
:1000E800A708031D79288711860183120313270B9C
:1000F8008028871510308600831203132708023AD8
:10010800031D882820308600831203132708033A2A
:10011800031D902830308600831203132708043A01
:10012800031DAE2840308600AE28831203138713C0
:100138000230D820BB20AE28831203138713023065
:10014800D820BB2083120313A611A61010108F010C
:100158008E01101483120313A618512856300F026B
:10016800031C5128A61410108F018E0151288312E8
:10017800031307170130D82083120313071308004D
:1001880083120313A2000230831681008312031323
:1001980081017D30831203130102031CCD288312D1
:1001A8000313A20BCA28080083120313A300A40197
:1001B80083120313230824020318F028A501FA3038
:1001C8008312031325020318EC280000A50AE3286C
:0A01D80083120313A40ADC280800B8
:02400E00D400DC
:00000001FF
